:1000000003308A006F2B00000A108A100A11820741
:1000100043346F34703479347234693467346834FB
:100020007434203432343034313434342034433472
:100030006C3469346E3474346F346E342034543418
:10004000753472346E3465347234203463346334FE
:1000500074342E346F3465346934403467346D340D
:10006000613469346C342E3463346F346D3400344D
:10007000A13480308318BD06C201C3013908C10014
:100080003D08C106380803192629C000A0003C0815
:1000900003192F29C0020319CC28031C8B283D0803
:1000A000C600C6173E08C5003F08C400C3010310C0
:1000B000C60CC50CC40CC30CC00B5628C11F63284A
:1000C000421443294210401042163B308400582904
:1000D0004212C11B7528401C8028C60CC50CC40CDC
:1000E000C30CA00A03193E298028C61B83280310CD
:1000F000C30DC40DC50DC60DA00303193E297528F7
:100100004217EB2842133908C100C11F8928C617BE
:100110003729C61337293C08C000A0003808C002A0
:100120003908C600C6173A08C5003B08C400C30119
:100130000310C60CC50CC40CC30CC00B9728C11F00
:10014000A428C2144329C2104010C2163F308400B4
:100150005829C212C11BB628401CC128C60CC50CA8
:10016000C40CC30CA00A03193E29C128C61BC4280D
:100170000310C30DC40DC50DC60DA00303193E2900
:10018000B628C217EB28C2133D08C100C11FCA28F8
:10019000C6173729C61337293D08C600C6173E08BB
:1001A000C5003F08C400C11FD928C6134215432902
:1001B0004211C30140103B3084005829C11B012962
:1001C0003908C100401CEB28C60CC50CC40CC30C7C
:1001D000A00A03193E29C31FFC28C40A031DFC28DA
:1001E000C50A031DFC28C60A031DFC28C60CC50C45
:1001F000C40CA00A03193E29421B8228C21BC32833
:1002000020298030C606C61F092943293D08C100A0
:1002100016293908C100C608031D1629C508031D83
:100220001629C408031D1629A0013729C61B202939
:100230000310C30DC40DC50DC60DA00B16293E2914
:10024000C11F2429C6173729C61337293C08A00027
:100250003D08C6003E08C5003F08C40037293808DD
:10026000A0003908C6003A08C5003B08C40046088B
:10027000A1004508A2004408A3007629A001A1011D
:10028000A201A3017629C301C409C509C609C3098E
:10029000C30A031D5129C40A031D5129C50A0319A4
:1002A000C60A42186228C218A3284219D82806296B
:1002B0000008C407031C6229C50A031D6229C60A77
:1002C0000319401484030008C507031C6A29C60AE1
:1002D0000319401484030008801F803AC6070318DE
:1002E0004014421A6828C21AA928DE2808003908D2
:1002F000C0003D08C006C01F822903110310B91BAE
:100300000314B5293908C0003C08C1003808C102EF
:1003100003199029C01FB5290308013A8300B529A4
:100320003D08C1003908C10203199C29C01FB52925
:100330000308013A8300B5293E08C1003A08C1020A
:100340000319A829C01FB5290308013A8300B5295C
:100350003F08C1003B08C1020319B429C01FB529D9
:100360000308013A8300B529031008008501033012
:10037000831685009501811771308F000F080030BA
:100380008312A1009200003083169200F030831295
:100390009505093098000F30A0008101813084005C
:1003A0000008F0390738800064000008F739A01908
:1003B000F039200480001F1383161F149F141F118F
:1003C0009F118312B8013808042000380319F72957
:1003D000B80AB9003908BA003A088400800803193D
:1003E000F329BA0AEC2939083A02A100E3292F3C83
:1003F000031D022A83161F169F121F1783129F17B1
:100400001F14092A83161F129F121F1383129F178E
:100410001F140030A1001F08F33921049F00900130
:100420000B138B138B1B112A64000130A600F430D0
:10043000A500A801A701AA01A90105113310B31055
:100440000030A1001F08F33921049F0064000F3021
:10045000A000A00B292A2C2A00009F14AE01AD0198
:10046000AC01AB01A90A0319AA0AB201B1011E30FD
:10047000B0008630AF00A90A0319AA0AA90A031915
:10048000AA0A2A08B9002908B8008E30A000390845
:10049000A1003808A200A301A108031D592A2208BF
:1004A000A100A2010830A002A108031D592AA00141
:1004B000612A0310A11B602AA20DA10DA003592AD5
:1004C000A11383103208BB003108BA003008B9000C
:1004D0002F08B8002308BF002208BE002108BD0075
:1004E0002008BC0039202308B2002208B1002108EE
:1004F000B0002008AF0083102E08BB002D08BA0002
:100500002C08B9002B08B8003208BF003108BE0023
:100510003008BD002F08BC0039202308AE00220897
:10052000AD002108AC002008AB00BB018030BA0050
:100530002030B9008630B8002E08BF002D08BE005C
:100540002C08BD002B08BC007721031CB92A3208F7
:10055000BB003108BA003008B9002F08B800BF014D
:100560008030BE002130BD008630BC0077210318EA
:10057000C02A1F1383161F109F101F159F1583126B
:10058000842B051685120800051285160800B40A8A
:100590000330B405B408031DCF2AC122D02AC422D7
:1005A00008003A30840000080319E72A0230A1004D
:1005B000BF30A0006400A00BDA2AA10BD82A963025
:1005C000A000A00BE12AE42A6400800BD62A0800D0
:1005D0000512851208000530B900DC30B800380873
:1005E00039040319192B3908013C031CFF2A031D88
:1005F000FD2A3808F33C031CFF2AC722112B3808B8
:10060000E83C031D092B3908033C031D092BC122BB
:10061000112B3808DC3C031D112B3908053C03194C
:10062000C42238080319B903B8030130BA00D12233
:10063000EF2AE822852B250826040319232B2508F9
:100640000319A603A50329082A0403192B2B29083B
:100650000319AA03A903270828040319332B270821
:100660000319A803A7038F2B2608003C0318422B6D
:10067000FF3A031D3F2B2508A93C0318422B4B30A2
:10068000BA00D1220430A1001F08F33921049F00D1
:1006900064000F30A000A00B4B2B4E2B0000051D5B
:1006A000562B0511E8224B30BA00D1229F149F1817
:1006B000572B1E08A30083161E088312B8002308B8
:1006C000B900023C03186D2BFF3A031D6B2B380851
:1006D000313C03186D2BB3146E2BB310E82B0308B9
:1006E0001F398300713083168F000F0883121F1388
:1006F00083161F109F101F119F110730831299003E
:10070000A401B4013710B629EB2A0030A1001F085C
:10071000F33921049F000130BA00D1221B2B371876
:10072000992B9F18912B83161E088312B5001E0863
:10073000B6009F14B318CA2B3608023C031CAD2B1D
:10074000031DA62B3508103C031CAD2B25082604E1
:10075000031DAC2B05153314BE2B3608013C0318C2
:10076000BE2BFF3A031DB82B3508273C0318BE2BC0
:10077000051133100130A600F430A500331CC52B41
:10078000C122AA011930A900C92B29082A0403197A
:10079000C422DE2B05113310AA08031DDD2B290806
:1007A000313C031CDD2BC72229082A04031DDC2B46
:1007B0000730AA00D030A900DE2BE8223710270826
:1007C0002804031DE92B1330A8008830A700342B20
:0607D0003714852B6300C5
:02400E00EC378D
:084000000200010005000400AC
:00000001FF
